:020000040000FA
:0200000087284F
:020008001228BC
:1000100054205820502036203120352020203020F8
:100020002E2031200800640085191328851D16280C
:100030000800640085191928FA30C9006400851980
:100040001928851919288519192885191928851934
:100050001928851919288519192885191928C90BEE
:100060001E28080084003130FF3E03183428083071
:10007000C5008001840A80019F149F183D281E0836
:10008000800783161E08831284038007840A0318DE
:10009000800AC50B3C2803300310800C8403800CBD
:1000A000840AFF3E031D4C2808001F1141303220F6
:1000B000C20CC10CC20CC10C4108C6001F15433054
:1000C0003220C40CC30CC40CC30C4308C700080086
:1000D000C80079200511AB306D286E28FF3E03184B
:1000E0006C28C80A732874280000C80B72280515EC
:1000F000003449307B287C28FF3E03187A2808000A
:10010000851D80280515851983280511080085019E
:100110000B306500831653309F0083126400810109
:10012000DF3062006400DC306200640007309A0057
:1001300081309F00C001552013201920802080208D
:10014000802080208020802013200515460868200C
:0C015000470868207920051155209D28E3
:02400E00DC3F95
:00000001FF
